:100000001AC034C033C032C031C030C02FC02EC07F
:100010002DC0FFC12BC032C029C028C027C026C0B8
:1000200025C024C023C0030B081C08080E000404CC
:10003000041F0404040011241FBECFE5D4E0DEBF7A
:10004000CDBF10E0A0E6B0E0E8ECF7E002C005901C
:100050000D92A636B107D9F710E0A6E6B0E001C0D0
:100060001D92A437B107E1F75ED0ACC3C9CF10929F
:100070006600109267001092680008951F920F9218
:100080000FB60F9211248F93EF93FF938CB180934F
:100090006900809168008830B8F4E0916600F0E073
:1000A0008CB1E459FF4F8083809168008F5F80930B
:1000B0006800809166008F5F809366008091660083
:1000C000883011F410926600FF91EF918F910F909C
:1000D0000FBE0F901F90189580916800882311F42F
:1000E000E0E016C0E0916700F0E0E459FF4FE081E6
:1000F00080916800815080936800809167008F5FD5
:100100008093670080916700883011F41092670037
:100110008E2F08955D9BFECF8CB908958091690064
:100120001092690008952F923F924F925F926F92C2
:100130007F928F929F92AF92BF92CF92DF92EF9277
:10014000FF920F931F93DF93CF9300D000D0CDB7D2
:10015000DEB7B89AC09883B7856083BF89B78160DE
:1001600089BF12BE1FD281D281E073D280EA9FE0A4
:100170000197F1F710BC83E389B988E98AB986E869
:1001800080BD789486E290E061E0B9D28EE290E0A2
:1001900062E0B5D28AE85DD281E061D280E690E08B
:1001A00094D280E0E8D18824992466247724CC2452
:1001B000DD241FE0A12EB12CB8EC2B2E312CA5E5AF
:1001C0004A2E19D2182F8BEC44D283E690E07DD2D0
:1001D0008A2DB1D1133021F40894A11CB11C05C0A3
:1001E000143019F40894A108B108CA14DB0410F003
:1001F000C09A01C0C098123011F500E05D9BFECF9F
:1002000020E52CB969DF182F109266001092670064
:10021000109268008AE81DD281E021D280E690E049
:1002200054D2812F8D52A7D184EF91E0F101319703
:10023000F1F70197D9F70F5F0A3001F704C01130C9
:1002400011F48824992455245D9BFECF4CB88091ED
:100250006C0090E09A83898380916D0090E09C838C
:100260008B831092660010926700109268008B8159
:100270009C8129813A81182F0027020F131F88EED5
:1002800093E0F1013197F1F70197D9F75D9BFECF2C
:100290004CB880916C0090E09A83898380916D00C6
:1002A00090E09C838B8310926600109267001092FE
:1002B00068008B819C8129813A81F82FEE27E20F1B
:1002C000F31F0E171F07C8F431E102361307A8F415
:1002D00081E1E236F80788F4CF01801B910B9C0185
:1002E00073E0220F331F7A95E1F7880F991F820F71
:1002F000931F6AE070E030D23B01E017F107C8F4C9
:1003000021E102361207A8F431E1E236F30788F45E
:10031000C8018E1B9F0B9C0153E0220F331F5A957F
:10032000E1F7880F991F820F931F6AE070E014D2E3
:100330003B018614970408F44301C40164E670E0AD
:100340000BD28B0180E885D1802F15D18CE287D12B
:1003500024E630E0029FC001039F900D129F900D94
:100360001124382D381B832F06D180E278D18DE6F9
:1003700076D18FE274D183E672D124E230E0829E9E
:10038000C001839E900D929E900D11246AE070E052
:10039000E3D17B0100E010E0C801B70124E630E0C2
:1003A00040E050E0EDD1690180EC53D18C2DC3D0F9
:1003B0008CE255D124E630E0C29EC001C39E900D70
:1003C000D29E900D1124A0E0B0E0E81AF90A0A0BC1
:1003D0001B0BC801B7012AE030E040E050E0D0D16B
:1003E000822FDDD080E23BD18BE639D18DE637D14B
:1003F0008FE235D188E633D184EF91E0F101319776
:10040000F1F70197D9F753943AE0531609F01CCF4E
:10041000D8CE1F920F920FB60F9211242F933F93B5
:100420004F935F936F937F938F939F93AF93BF93FC
:10043000EF93FF93BED0FF91EF91BF91AF919F914A
:100440008F917F916F915F914F913F912F910F907D
:100450000FBE0F901F901895EF92FF920F931F936E
:100460009C0168EE73E078D1182F092FC90168EE5E
:1004700073E072D1662311F480E302C0862F805DA1
:10048000EED0812F902F64E670E066D1F82EE92E31
:10049000812F902F64E670E05FD1662311F480E332
:1004A00002C0862F805DDBD08F2D9E2D6AE070E02C
:1004B00053D1362F8F2D9E2D6AE070E04DD1182F2D
:1004C000332311F480E302C0832F805DC8D0812FD5
:1004D000805DC5D01F910F91FF90EF9008950F930D
:1004E0001F939C0164E670E037D1182F092FC901D2
:1004F00064E670E031D1662311F480E302C0862FF8
:10050000805DADD0812F902F6AE070E025D1362F2D
:10051000812F902F6AE070E01FD1182F332311F440
:1005200080E302C0832F805D9AD0812F805D97D0B9
:100530001F910F9108951F93282F64E601D1192F61
:10054000822FFED0882311F480E301C0805D87D024
:10055000812F6AE0F5D0282F812FF2D0192F222386
:1005600011F480E302C0822F805D79D0812F805DFD
:1005700076D01F9108951F93282F6AE0E1D0382F7D
:10058000822FDED0192F332311F480E302C0832F92
:10059000805D65D0812F805D62D01F910895805D60
:1005A0005ED0089584B3807F84BB85B38F6085BBA4
:1005B0000895989902C091E00BC09A9902C093E007
:1005C00007C0999902C092E003C09B9911C094E0C2
:1005D00080916B00873420F08EE380936B0005C020
:1005E0008F5F80936B00843029F490936A000895A4
:1005F00010926B00089580916A0010926A0008952D
:1006000080936A0008959AE69A95F1F7C39892B399
:10061000807F9F70982B92BBC19A85E08A95F1F7F5
:10062000C198089592B3282F207F9F70292B22BB59
:10063000C19A25E0922F9A95F1F7C19892B38295CD
:10064000807F9F70982B92BBC19A2A95F1F7C19831
:1006500008959AE69A95F1F7C398E4DF08959AE62B
:100660009A95F1F7C39ADEDF08950F931F9381B334
:10067000806F81BBBB9ABA9AB99A80E991E028EC65
:1006800030E0F9013197F1F70197D9F780E3BBDF4B
:1006900080E29EE40197F1F780E3B5DF00EA1FE016
:1006A000C8010197F1F780E3AEDF88E2ACDF88E2B2
:1006B000D0DF8CE0CEDF81E0CCDFC8010197F1F71D
:1006C00086E0C7DF1F910F910895CF93DF93EC0170
:1006D00002C02196C4DF88818823D9F7DF91CF91AA
:1006E0000895CF93DF93EC0104C0FE01849121961D
:1006F000B6DF88818823C9F7DF91CF9108950F93E2
:100700001F93CF93DF938C01862F90E087709070BA
:1007100023E0880F991F2A95E1F780649ADFC0E0F3
:10072000D0E0F801EC0FFD1FE4918E2F98DF2196A9
:10073000C830D105B1F7DF91CF911F910F91089586
:10074000991B79E004C0991F961708F0961B881F23
:100750007A95C9F780950895AA1BBB1B51E107C084
:10076000AA1FBB1FA617B70710F0A61BB70B881F41
:10077000991F5A95A9F780959095BC01CD010895D0
:10078000A1E21A2EAA1BBB1BFD010DC0AA1FBB1F95
:10079000EE1FFF1FA217B307E407F50720F0A21B07
:1007A000B30BE40BF50B661F771F881F991F1A9474
:1007B00069F760957095809590959B01AC01BD019E
:0807C000CF010895F894FFCF6A
:0607C800433D004C3D0022
:00000001FF
